:020000040000FA
:06000000F6EF00F0120013
:0A0006000100180200008B0000004A
:0400100001000000EB
:0C001400060EF66E000EF76E000EF86E81
:1000200000010900F550856F0900F550866F03E166
:10003000856701D03DD00900F550806F0900F5506B
:10004000816F0900F550826F09000900F550E96ED3
:100050000900F550EA6E090009000900F550836FA8
:100060000900F550846F09000900F6CF87F0F7CF3B
:1000700088F0F8CF89F080C0F6FF81C0F7FF82C01A
:10008000F8FF0001835302E1845307E00900F550B3
:10009000EE6E8307F8E28407F9D787C0F6FF88C0C1
:1000A000F7FF89C0F8FF00018507000E865BBFD708
:0200B00012003C
:0E00B200D9CFE6FFDACFE6FFE1CFD9FFE2CFEC
:1000C000DAFFAC6AAB6AFD0EDBB0AC88DBA202D013
:1000D000AC8CAB8CDBB4AC8EDBA602D0AB8801D091
:1000E000AB8ADBA802D0AC8401D0AC949E98DBAC88
:1000F00002D09D8A01D09D9A9E9ADBAE02D09D8847
:1001000001D09D98FB0EDB50AF6EAC8AAB8E949CF9
:10011000948EAC50100B04E0AC50800B01E1948C39
:0C012000E552E5CFDAFFE7CFD9FF12006F
:04012C00D9CFE6FF42
:10013000E1CFD9FF040EE126DE6ADD6A020EDB6A3A
:10014000030EDB6A190EE66EE66A3C0EE66E59ECAB
:1001500000F0E552E552E5528BC0E6FFDFEC00F01F
:10016000E5520A0EE66EC8EC00F0E55200018B2B5A
:10017000380E8B5D02E1300E8B6FEED7040EE15C22
:1001800002E2E16AE552E16EE552E7CFD9FF1200E3
:10019000FF0EE350036EEF0E01D0F30EE76EE72E75
:1001A000CFEF00F00C0E026EE76AE72ED5EF00F0FD
:0E01B000022ED4EF00F0032ECDEF00F012006F
:0201BE00D9CF97
:1001C000E6FFDACFE6FFE1CFD9FFE2CFDAFFACAC52
:1001D00004D0AC9000018AB3AC80FD0EDB50AD6E54
:0C01E000E552E5CFDAFFE7CFD9FF1200AF
:0401EC0015EE00F01C
:1001F00025EE00F0F86A019C0AEC00F00BEC01F02F
:0802000096EC00F0FBD71200A0
:0802080000EE00F00F0EEE6A9B
:06021000EA62FDD71200B6
:020216001200D4
:0102180031B4
:00000001FF
